:0600000002356302006BF3
:03000B0002006B85
:0300130002006B7D
:03001B0002006B75
:0300230002006B6D
:03002B0002006B65
:0300330002006B5D
:03003B0002006B55
:0300430002006B4D
:03004B0002006B45
:0300530002006B3D
:03005B0002006B35
:0300630002006B2D
:01006B003262
:0900800002006B0002006B00029B
:08008900006B0002006B000295
:08009100006B0002006B00028D
:08009900006B0002006B000285
:0800A100006B0002006B00027D
:0800A900006B0002006B000275
:0700B100006B0002006B0070
:0901000002006B0002006B00021A
:08010900006B0002006B000214
:08011100006B0002006B00020C
:08011900006B0002006B000204
:08012100006B0002006B0002FC
:08012900006B0002006B0002F4
:08013100006B0002006B0002EC
:08013900006B0002006B0002E4
:08014100006B0002006B0002DC
:08014900006B0002006B0002D4
:08015100006B0002006B0002CC
:08015900006B0002006B0002C4
:08016100006B0002006B0002BC
:08016900006B0002006B0002B4
:08017100006B0002006B0002AC
:07017900006B0002006B00A7
:0801800078B0E84403600C793B
:0C01880004903800E4F0A3D8FCD9FAD0B1
:0E01940083D082F6D8FDC082C083758200221F
:0CE0000012010002000000404705020071
:06E00C0000010102060103
:0AE012000A060002000000400100B1
:0EE01C0009023B00030100C0000904000002DD
:0EE02A00FE030104070502020002000705863E
:0EE03800020002000904010000FFFFFF0309BF
:0EE0460004020000FE010105092101F4014061
:03E05400000001C8
:0CE0580012010002000000404705020019
:06E06400000101020601AB
:0AE06A000A06000200000040010059
:0EE0740009023200030100C00009040000028E
:0EE08200FE03010407050202400000070586A8
:0EE09000024000000904010000FFFFFF030929
:08E09E0004020000FE0101056F
:0CE0A600120100010000004047050300CB
:06E0B2000001010206015D
:0EE0B80009021200010100C00009040000006E
:04E0C600FE01020550
:09E0CA00092101F40140000001EC
:01E0D3000745
:02E0D400E2E088
:02E0D600E8E080
:02E0D80008E15D
:02E0DA001CE147
:02E0DC003EE123
:02E0DE005AE105
:02E0E0007CE1E1
:06E0E20006030000090422
:0EE0E80020034D006900630072006F004C00C1
:0EE0F6006100620020004200460048002D003C
:04E10400540049007A
:0EE1080014034700450043004B004F00330056
:06E1160043004F004D0024
:0EE11C00220343006F006D006D0061006E0075
:0EE12A006400200026002000530074006100F5
:06E1380074007500730085
:0EE13E001C0355005300420054004D004300E6
:0EE14C00200055005300420034003800380017
:0EE15A0022034700450043004B004F003300F6
:0EE1680043004F004D002000450045005000D0
:06E1760052004F004D00B5
:02E17C0012038C
:0EE17E0033002E00310034003100350039002E
:02E18C0033005E
:0A01A200AA82AB09903800EBF0AB25
:0701AC0008903801EBF0752B
:0301B3004F007585
:0301B60050387549
:0C01B90051028A82C002122C68E582D03C
:0601C500027003F5822226
:0401CB00850A4F85CD
:0301CF000B50854D
:0501D2000C518A8202BD
:0201D7002BA853
:0A01D900AA82C374FF950D743F95D0
:0701E3000E5004758200229A
:0701EA00E511700302029F02
:0A01F100AB117C00EB250DFBEC3593
:0801FB000EFC74C0550DFDAEB1
:0C0203000E74402DFDE43EFEC3ED9BEEAA
:0C020F009C500E743F550DFB7C007440A9
:05021B00C39BFB800CF9
:0A02200074C025114004AB118002E8
:02022A007B4017
:08022C00AC0E903802ECF0ACBE
:0A0234000D7D00903803ECF07C0013
:0C023E00C3EC9B501E74022C2402FDE453
:0A024A003438FEEC250FF582E43590
:0C02540010F583E0FF8D828E83F00C809B
:01026000DDC0
:04026100754F02755E
:06026500503874022BF575
:0C026B00518A82C002C003122C68E58298
:09027700D003D0027003F58222CD
:0A028000E511C39BF5117C00EB258E
:05028A000DF50DEC353F
:09028F000EF50E900008C00212E9
:070298003508D0020201EA63
:04029F007582012241
:0E02A300903844E4F0903845F0A3F0A3F0A3A7
:0E02B100F0903849E4F090384AF0A3F0A3F042
:0E02BF00A3F090384EE4F0A3F0A3F0A3F07586
:0602CD001201751301751A
:0602D30014807515007592
:0602D9001600751700225B
:0E02DF00AA82AB83ACF0123547FD74012AFEF3
:0E02ED00E43BFF8C008E828F8388F012354731
:0902FB00FE5D6005430520800250
:020304007D007A
:0E0306008A828B838CF0ED1233B674022AFFCC
:0E031400E43BF88C018F82888389F012354714
:0E032200FD74032AFAE43BFB8A828B838CF085
:0E033000123547FE74BF5DFA8A0574BF5E5A2F
:0D033E00600D4305408F82888389F0ED1229
:02034B0033B6C7
:03034D008D82227C
:0D03500090E6B8E0FA530280BA8002800304
:03035D000206583D
:0A03600090E6B9E0FABA0102804508
:06036A00BA0203020425A3
:06037000BA030302049130
:06037600BA04030204F8C2
:06037C00BA05030205644E
:06038200BA06030205C9E2
:06038800BA07030205E4C0
:06038E00BA400302060262
:06039400BA800302061E00
:06039A00BAA00302066F89
:0603A000BAA10302064CA5
:0603A600BAA2030206509A
:0303AC00020654F2
:0903AF007401B51A0B75120175F9
:0703B800130112199E804998
:0E03BF00903844E0FA90E6BAE0FBEAB5033865
:0A03CD0075120175130190E6047427
:0E03D70080F00090E6047482F00090E6497415
:0E03E50082F00090E6497482F00090E64974C0
:0E03F30082F00090E6497482F00090E604E487
:04040100F000800384
:03040500751281EC
:0C04080090E740E512F0903844E0FA90D4
:0E041400E741F090E68AE4F090E68B7402F087
:0304220002066F60
:0A04250075120190E740E512F09017
:0D042F00E741E4F090E742F090E743F090E1
:0E043C00384AE0FAA3E0A3E0A3E090E744EA28
:0E044A00F090384AE0A3E0FBA3E0A3E08B02B1
:0E04580090E745EAF090384AE0A3E0A3E0FC0C
:0E046600A3E08C0290E746EAF090384AE0A34B
:0E047400E0FBA3E0FCA3E0FD8D0290E747EA69
:0D048200F090E68AE4F090E68B7408F0023A
:02048F00066FF6
:090491007401B51A2675120175FB
:0C049A00130112199E90E6047480F0001B
:0E04A60090E6047486F00090E6487486F0003C
:0804B40090E604E4F000801F53
:0E04BC00903844E0FA90E6BAE0FBEAB5030E91
:0904CA0075120175130174EF5560
:0504D30016F516800380
:0304D80075128119
:0C04DB0090E740E512F090E6BAE0FA90DD
:0E04E700E741F090E68AE4F090E68B7402F0B4
:0304F50002066F8D
:0A04F80075120190E740E512F09044
:0D050200E741E4F090E742F090E743F0900D
:0E050F00384EE0FAA3E0A3E0A3E090E744EA50
:0E051D00F090384EE0A3E0FBA3E0A3E08B02D9
:0E052B0090E745EAF090384EE0A3E0A3E0FC34
:0E053900A3E08C0290E746EAF090384EE0A373
:0E054700E0FBA3E0FCA3E0FD8D0290E747EA95
:0D055500F090E68AE4F090E68B7408F00266
:02056200066F22
:0905640075120175130174EF55C5
:06056D0016F5167401B53D
:060573001A09121A0775B7
:050579001A001214D36A
:0E057E0090E6047480F00090E6047482F000B1
:0E058C0090E6047486F00090E6497482F00058
:0E059A0090E6497482F00090E6497482F00009
:0E05A80090E6497482F00090E604E4F00090C2
:0B05B600E740E512F090E68AE4F090C8
:0805C100E68B7401F002066FE5
:0A05C90075120190E740E512F09072
:0E05D300E741E4F090E68AF090E68B7402F0C7
:0305E10002066FA0
:0605E4007512017A967BFE
:0905EA003590E6B3EBF07A967B44
:0C05F300357B007C007D0090E6B4EAF04F
:0305FF0002066F82
:0C060200758206121B8475120190E740FF
:0C060E00E512F090E68AE4F090E68B74B0
:04061A0001F080511A
:0A061E0075120190E740E512F0901C
:0E062800E6BAE090E741F090001475F0401241
:0E06360002DFAA8290E742EAF090E68AE4F042
:0806440090E68B7403F08023A3
:04064C007582002291
:04065000758200228D
:040654007582002289
:0D06580090E6B8E0FA20E70B90E6B9E075F7
:06066500128075820022E4
:04066B007582002272
:04066F00758201226D
:0E359600010000010400000000000000000120
:0A35A400000000000000000000001D
:0E067300AA8275F00AEA84A9F0EAC39975F02C
:0D0681000A84FA75F00A84E5F0FC7027ADDC
:04068E004FAE50AF6C
:0C06920051743029F88D828E838FF01295
:07069E0033B60DBD00010E93
:0E06A5008D828E838FF0740A1233B675820236
:0106B3002224
:0E06B400EAC39C75F00A8475F00A84E5F0FA3A
:0706C200703DAD4FAE50AFDB
:0B06C9005174302C8D828E838FF01254
:0E06D40033B674012DFAE43EFC8F0074302919
:0E06E2008A828C8388F01233B674022DFDE4F8
:0E06F0003EFE8D828E838FF0740A1233B67533
:0306FE0082032252
:05070100AB4FAD50AE4E
:0B0706005174302A8B828D838EF0121C
:0E07110033B674012BFAE43DFF8E0074302CD9
:0E071F008A828F8388F01233B674022BFAE4BC
:0E072D003DFC8E077430298A828C838FF01277
:0E073B0033B674032BFBE43DFD8B828D838E61
:0A074900F0740A1233B67582042220
:0807530085824F85835085F07B
:08075B00517552007E007F0081
:03076300BF0400D0
:0A076600505CEF254FFDE43550FA1A
:0C077000AB518D828A838BF0123547FA62
:03077C00BA300090
:0C077F004014EA24C6400FE55275F00A51
:0A078B00A4FBEA24D02BF552802ACB
:09079500EE254FFAE43550FBACEF
:0C079E00518A828B838CF0123547FABA26
:0407AA000A028003BC
:0307AE00EA7004EA
:0407B10085528222C9
:0A07B50074104514F514758200223B
:0507BF000F8F06809F72
:0A07C40074104514F514758200222C
:0807CE0085825285835385F0FA
:0407D60054AD4FAE21
:0507DA0050AF51780052
:0E07DF008D828E838FF01235477A0024FEF94A
:0E07ED00EA34FFFA88037C00C3EB99EC6480C9
:0D07FB008AF063F08095F05038E8C31325B4
:0508080052F555E43536
:04080D0053F55685C4
:0A081100545774022BFBE43CFCEB8F
:0E081B002DFBEC3EFC8F028B828C838AF01248
:070829003547FB8555828570
:0608300056838557F0120B
:0608360033B6080880A3A0
:0D083C00E8C313FA8A037C000BBB00010C1B
:09084900EB2552FBEC3553FCAD2C
:0C085200548B828C838DF0E41233B6EAE4
:08085E002552FAE43553FBAC0E
:08086600548A828B838CF0227E
:0E086E00AA82AB83ACF0123547FDA3123547CA
:08087C00FEA3123547FF7800CE
:0A088400C3E895255069E82522F528
:05088E0026E43523F50E
:0308930027852492
:0C089600288D828E838FF0123547F5828A
:0E08A200C002C003C004C005C006C007C000ED
:0E08B00012351BE582D000D007D006D005D04F
:0E08BE0004D003D002600F8D828E838FF01263
:0808CC003547F9430120800AC1
:0A08D4008D828E838FF0123547F9F4
:0708DE008526828527838532
:0B08E50028F0E91233B60DBD00010E33
:0308F000088091EC
:0D08F3008A828B838CF0ED1233B6A3EE12D7
:0E09000033B6A3EF1233B674062AFDE43BFEB5
:0B090E008C078D828E838FF0E5221293
:0609190033B6A3E5231232
:06091F0033B6A3E524122B
:0C09250033B674092AFAE43BFBE52525F3
:0709310022FDE43523FEAFB7
:0C093800248A828B838CF0ED1233B6A36E
:0A094400EE1233B6A3EF1233B685AE
:06094E002282852383854F
:0309540024F0226A
:0809570085822C85832D85F0BB
:08095F002E7406252CFDE43581
:050967002DFEAF2E750E
:03096C002252759F
:03096F00233875B5
:06097200240075250C8530
:060978002C82852D838511
:0C097E002EF0C005C006C00712086EAACB
:0E098A0082AB83ACF0D007D006D0058D828EF4
:0E099800838FF0EA1233B6A3EB1233B6A3EC52
:0A09A6001233B67406252CFAE4356E
:0A09B0002DFBAC2E8A828B838CF0A5
:0709BA00123547F52FA312CF
:0609C1003547F530A312DA
:0509C7003547F5318504
:0609CC002F8285308385B7
:0B09D20031F0123547FDBD2A02800302
:0309DD00020FC83E
:0A09E0007401252FFDE43530FEAF51
:0C09EA00318A828B838CF0ED1233B6A3AF
:0A09F600EE1233B6A3EF1233B68DF4
:040A00004F8E508F36
:060A040051755203E4F5F8
:0C0A0A00539035AE75F080C002C003C0F0
:0E0A160004122A02E5828583F0D004D003D0BA
:0A0A24000245F0700BF514F516758D
:060A2E0013017582012294
:0C0A34008A828B838CF0123547F54FA3AB
:070A4000123547F550A31227
:050A47003547F5517573
:060A4C005203E4F5539093
:0E0A520035B275F080C002C003C004122A0243
:0E0A6000E5828583F0D004D003D00245F0601B
:040A6E0003020B363E
:0E0A72008A828B838CF0123547FDA312354724
:0E0A8000FEA3123547FF74032DFDE43EFE8AEF
:0E0A8E00828B838CF0ED1233B6A3EE1233B6DA
:0E0A9C00A3EF1233B68A828B838CF01235479B
:070AAA00F532A3123547F5F8
:060AB10033A3123547F5E6
:0C0AB700348D828E838FF0123547FDBD18
:0A0AC300201F74012532FDE43533D5
:0C0ACD00FEAF348D828E838FF012075331
:0A0AD900E582F51575130175820121
:010AE30022F0
:070AE4008532828533838512
:0A0AEB0034F0123547FDBD3F3EAA6E
:040AF50029AB2AAC53
:070AF9002B8A3574012BF577
:040B0000368C378573
:050B040015828A4F8BF1
:040B0900508C5112A9
:0A0B0D000673AD827E0085358285F7
:070B170036838537F0ED1273
:0A0B1E0033B6A3EE1233B67410458F
:040B280016F5167533
:060B2C0013017582012295
:040B320075820022A6
:0C0B36008A828B838CF0123547F54FA3A8
:070B4200123547F550A31224
:050B49003547F5517570
:060B4E005204E4F553908F
:0E0B540035B675F080C002C003C004122A023C
:0E0B6200E5828583F0D004D003D00245F07008
:060B700041AA29AB2AACEA
:070B76002B8A3274012BF5FC
:040B7D00338C3485FC
:050B810014828A4F8B75
:040B8600508C51122C
:0A0B8A000673AD827E00853282857D
:070B940033838534F0ED12FC
:0A0B9B0033B6A3EE1233B674104512
:040BA50016F51675B6
:090BA9001400751301758201228C
:0C0BB2008A828B838CF0123547F54FA32C
:070BBE00123547F550A312A8
:050BC5003547F55175F4
:060BCA005204E4F5539013
:0E0BD00035BB75F080C002C003C004122A02BB
:0E0BDE00E5828583F0D004D003D00245F0609C
:040BEC0003020CFFF5
:050BF000AA29AB2AACAC
:0A0BF5002B90E066E075F002A424E6
:0A0BFF00D4F58274E035F0F583E0D0
:090C0900FDA3E0FE8D4F8E507535
:0C0C120051008A828B838CF01207CEAA5E
:0E0C1E0082AB83ACF0742C1233B674012AF54D
:060C2C0035E43BF5368CB7
:0A0C32003790E067E075F002A4249B
:0A0C3C00D4F58274E035F0F583E092
:090C4600FDA3E0FE8D4F8E5075F8
:060C4F005100853582858D
:060C550036838537F01222
:0E0C5B0007CEAA82AB83ACF0742C1233B60A1B
:040C6900BA00010BC1
:0C0C6D0090E068E075F002A424D4F58249
:0C0C790074E035F0F583E0FDA3E0FE8D93
:040C85004F8E5075C9
:0C0C890051008A828B838CF01207CEADE4
:040C950029AE2AAFAB
:030C99002B754F69
:030C9C00C07550D0
:0A0C9F00357551808D828E838FF031
:060CA900122CE1AD29AEA2
:040CAF002AAF2B75C8
:030CB3004FC275B8
:030CB60050357541
:0C0CB90051808D828E838FF0122CE1AAF6
:040CC50029AB2AAC81
:070CC9002B8A3274012BF5A8
:0A0CD000338C348A828B838CF0127F
:0A0CDA00352FAD82AE83853282858E
:070CE40033838534F0ED12AB
:080CEB0033B6A3EE1233B67517
:070CF300130174104516F512
:050CFA001675820122C5
:0C0CFF008A828B838CF0123547F54FA3DE
:070D0B00123547F550A31259
:050D12003547F55175A5
:060D17005203E4F55390C5
:0E0D1D0035C775F080C002C003C004122A0260
:0E0D2B00E5828583F0D004D003D00245F0604D
:040D390003020DB5EF
:0E0D3D008A828B838CF0123547FDA312354756
:0E0D4B00FEA3123547FF74032DFDE43EFE8A21
:0E0D5900828B838CF0ED1233B6A3EE1233B60C
:0E0D6700A3EF1233B68D828E838FF0123547C4
:090D7500FDBD3F32AD29AE2AAFED
:0C0D7E002B8D828E838FF074311233B6FF
:0D0D8A0074012EFE8D828E838FF074011295
:080D970033B6A3E41233B67574
:070D9F00130174104516F565
:050DA600167582012218
:0A0DAB00751801751301758201220D
:0C0DB5008A828B838CF0123547F54FA327
:070DC100123547F550A312A3
:050DC8003547F55175EF
:060DCD005203E4F553900F
:0E0DD30035CB75F080C002C003C004122A02A6
:0E0DE100E5828583F0D004D003D00245F07087
:0A0DEF001A740C252CFDE4352DFECE
:0B0DF900AF2E8D828E838FF0740112EC
:060E040033B675820122E5
:0C0E0A008A828B838CF0123547F54FA3D1
:070E1600123547F550A3124D
:050E1D003547F5517599
:060E22005203E4F55390B9
:0E0E280035CF75F080C002C003C004122A024C
:0E0E3600E5828583F0D004D003D00245F06041
:040E440003020F0690
:0E0E48008A828B838CF0123547FDA31235474A
:0E0E5600FEA3123547FF74032DFDE43EFE8A15
:0E0E6400828B838CF0ED1233B6A3EE1233B600
:0E0E7200A3EF1233B68A828B838CF0123547C1
:070E8000F535A3123547F51B
:060E870036A3123547F509
:0C0E8D00378D828E838FF0123547FDBD3B
:0A0E9900201F74012535FDE43536F5
:0C0EA300FEAF378D828E838FF012075354
:0A0EAF00E582F51775130175820145
:010EB9002216
:070EBA008535828536838532
:0A0EC10037F0123547FDBD3F38AA97
:040ECB0029AB2AAC79
:070ECF002B8A3274012BF5A0
:040ED600338C3485A0
:050EDA0017828A4F8B16
:040EDF00508C5112D0
:0A0EE3000673AD827E008532828521
:070EED0033838534F0ED12A0
:080EF40033B6A3EE1233B6750C
:060EFC00130175820122C2
:040F020075820022D2
:0C0F06008A828B838CF0123547F54FA3D4
:070F1200123547F550A31250
:050F19003547F551759C
:060F1E005204E4F55390BB
:0E0F240035D375F080C002C003C004122A024B
:0E0F3200E5828583F0D004D003D00245F07034
:060F400050AA29AB2AAC07
:070F46002B8A3274012BF528
:040F4D00338C34901D
:0E0F5100001475F040C002C003C0041202DF9D
:0A0F5F00D004D003D0028A4F8B505B
:0A0F69008C51120673AD827E0085E4
:060F730032828533838504
:090F790034F0ED1233B6A3EE12C0
:080F820033B67513017410452C
:070F8A0016F5167582012225
:0C0F91008A828B838CF0123547F54FA349
:070F9D00123547F550A312C5
:050FA4003547F5517511
:060FA9005203E4F5539031
:0E0FAF0035D875F080122A02E5828583F04560
:070FBD00F0700475820122AF
:040FC4007582002210
:040FC800852F4F859D
:030FCC003050851D
:030FCF0031517528
:060FD2005205E4F5539006
:0E0FD80035DC75F080C002C003C004122A028E
:0E0FE600E5828583F0D004D003D00245F06090
:040FF4000302117F64
:0E0FF8008A828B838CF0123547FDA312354799
:0E100600FEA3123547FF74052DFDE43EFE8A61
:0E101400828B838CF0ED1233B6A3EE1233B64E
:08102200A3EF1233B68D4F8ECF
:04102A00508F51751D
:06102E005204E4F55390AA
:0E10340035E275F080C002C003C004122A022B
:0E104200E5828583F0D004D003D00245F06033
:041050000302110E78
:08105400E51430E539AD29AEC9
:04105C002AAF2B7517
:031060004FE775E2
:0310630050357590
:0C10660051808D828E838FF012297CADAA
:07107200297401252AFEAFDD
:0C1079002B8D828E838FF074161233B61C
:0A108500A3E41233B674DF5514F52E
:03108F0014806F5B
:08109200E51430E439AD29AE8C
:04109A002AAF2B75D9
:03109E004FFE758D
:0310A10050357552
:0C10A40051808D828E838FF012297CAD6C
:0710B000297401252AFEAF9F
:0C10B7002B8D828E838FF074181233B6DC
:0A10C300A3E41233B674EF5514F5E0
:0310CD001480315B
:0510D000AD29AE2AAFBE
:0310D5002B754F29
:0310D80017755039
:0A10DB00367551808D828E838FF0F0
:0810E50012297CAD29740125DC
:0A10ED002AFEAF2B8D828E838FF058
:0A10F700740E1233B6A3E41233B6F0
:0811010075130174104516F589
:051109001675820122B1
:0C110E008A828B838CF0123547F54FA3CA
:07111A00123547F550A31246
:051121003547F5517592
:061126005205E4F55390B0
:0E112C00362675F080122A02E5828583F04592
:08113A00F0703EAD29AE2AAFB2
:031142002B754FBB
:031145002C7550B6
:0A114800367551808D828E838FF082
:0811520012297CAD297401256E
:0A115A002AFEAF2B8D828E838FF0EA
:0B11640074071233B6A3E41233B67513
:07116F00130174104516F591
:05117600167582012244
:04117B007582002257
:0C117F008A828B838CF0123547F54FA359
:07118B00123547F550A312D5
:051192003547F5517521
:061197005205E4F553903F
:0E119D00363475F080C002C003C004122A026E
:0E11AB00E5828583F0D004D003D00245F060C9
:0411B9000302137C9E
:0E11BD008A828B838CF0123547FDA3123547D2
:0E11CB00FEA3123547FF74052DFDE43EFE8A9B
:0E11D900828B838CF0ED1233B6A3EE1233B688
:0811E700A3EF1233B68D4F8E09
:0411EF00508F517557
:0611F3005205E4F55390E3
:0E11F900363A75F080C002C003C004122A020C
:0E120700E5828583F0D004D003D00245F0705C
:0A1215001A740C252CFDE4352DFEA3
:0B121F00AF2E8D828E838FF0740512BD
:06122A0033B675820122BB
:0C1230008A828B838CF0123547F54FA3A7
:07123C00123547F550A31223
:051243003547F551756F
:061248005205E4F553908D
:0E124E00364075F080C002C003C004122A02B0
:0E125C00E5828583F0D004D003D00245F07007
:0A126A001A740C252CFDE4352DFE4E
:0B127400AF2E8D828E838FF07403126A
:06127F0033B67582012266
:0C1285008A828B838CF0123547F54FA352
:07129100123547F550A312CE
:051298003547F551751A
:06129D005203E4F553903A
:0E12A300364675F080C002C003C004122A0255
:0E12B100E5828583F0D004D003D00245F070B2
:0A12BF001A740C252CFDE4352DFEF9
:0B12C900AF2E8D828E838FF074021216
:0612D40033B67582012211
:0C12DA008A828B838CF0123547F54FA3FD
:0712E600123547F550A31279
:0512ED003547F55175C5
:0612F2005205E4F55390E3
:0E12F800364A75F080C002C003C004122A02FC
:0E130600E5828583F0D004D003D00245F0705C
:0A1314001A740C252CFDE4352DFEA3
:0B131E00AF2E8D828E838FF0740412BE
:0613290033B675820122BB
:0C132F008A828B838CF0123547F54FA3A7
:07133B00123547F550A31223
:051342003547F551756F
:061347005204E4F553908E
:0E134D00365075F080122A02E5828583F04545
:0A135B00F0701A740C252CFDE43527
:0A1365002DFEAF2E8D828E838FF0D7
:09136F0074061233B675820122E6
:041378007582002258
:0C137C008A828B838CF0123547F54FA35A
:07138800123547F550A312D6
:05138F003547F5517522
:061394005204E4F5539041
:0E139A00365575F080C002C003C004122A024E
:0E13A800E5828583F0D004D003D00245F060CA
:0413B600030214CF4B
:0E13BA008A828B838CF0123547FDA3123547D3
:0E13C800FEA3123547FF74042DFDE43EFE8A9D
:0E13D600828B838CF0ED1233B6A3EE1233B689
:0813E400A3EF1233B68D4F8E0A
:0413EC00508F517558
:0613F0005205E4F55390E4
:0E13F600365A75F080C002C003C004122A02ED
:0E140400E5828583F0D004D003D00245F0705D
:0A1412001A740C252CFDE4352DFEA4
:0B141C00AF2E8D828E838FF0740912BA
:0614270033B675820122BC
:0C142D008A828B838CF0123547F54FA3A8
:07143900123547F550A31224
:051440003547F5517570
:061445005204E4F553908F
:0E144B00366075F080C002C003C004122A0291
:0E145900E5828583F0D004D003D00245F07008
:0A1467001A740C252CFDE4352DFE4F
:0B147100AF2E8D828E838FF074081266
:06147C0033B67582012267
:0C1482008A828B838CF0123547F54FA353
:07148E00123547F550A312CF
:051495003547F551751B
:06149A005204E4F553903A
:0E14A000366575F080122A02E5828583F045DC
:0A14AE00F0701A740C252CFAE435D6
:0A14B8002DFBAC2E8A828B838CF092
:0914C20074071233B67582012291
:0414CB007582002204
:0414CF007582002200
:0435AE00636C7300D7
:0435B20065736500D8
:0535B6006573723F0087
:0535BB0069646E3F0091
:0235C0002C00DD
:0535C200302E330A0069
:0435C7006F706300BE
:0435CB0072737400A3
:0435CF0073726500AE
:0535D3007374623F006B
:0435D80077616900AE
:0635DC00737973743A00DC
:0535E2006572723F005C
:0E35E7002D3130302C2022436F6D6D616E64EB
:0935F500206572726F72220A0057
:0E35FE002D3230302C202245786563757469BB
:0B360C006F6E206572726F72220A0060
:0E361700302C20224E6F206572726F72220AD4
:0136250000A4
:06362600766572733F009F
:08362C00313939392E300A0052
:06363400667067613A00B8
:06363A00636F6E662000C4
:06364000747970653F0083
:0436460069643F0074
:06364A00646F6E653F0095
:053650006461746100DB
:053655006D656D3A00F7
:06365A00646174612000B0
:0536600064656C200010
:053665006361743F00E9
:0814D30090E60174E0F0002234
:0814DB0085825485835585F0DC
:0514E30056755700756D
:0514E8005800AF51A8FF
:0514ED0052A953E4F5D3
:0714F2005BF55C74022FF5AD
:0614F9005DE438F55E8998
:0914FF005F74032FF560E438F579
:05150800618962E4F5B9
:03150D0059F55A33
:06151000C3E559954FE50B
:061516005A95504003024B
:02151C00163C7B
:0A151E00C3E5589557505DC007C0A3
:0915280000C001AB580558EB2589
:0715310060FBE43561FCAE34
:0415380062E55925EA
:05153C0054FAE55A35E8
:0A15410055FDAF568A828D838FF0AE
:0E154B00123547FA8B828C838EF01233B6E590
:0815590057B55804740180012C
:01156100E4A5
:0B156200D001D000D007700302162B50
:0C156D008F82888389F0E55B1233B6A3FF
:09157900E55C1233B67582012213
:07158200E558702DE5592525
:0515890054FAE55A359B
:0A158E0055FBAC568A828B838CF06B
:08159800123547FA855D8285DA
:0615A0005E83855FF0127E
:0B15A6003547FBEAB50306755801024B
:0215B100162BF7
:0815B3007401B55821E559252A
:0515BB0054FAE55A3569
:0A15C00055FBAC568A828B838CF039
:0A15CA00123547700575580280576E
:0515D400755800805273
:0915D9007402B5584D755800E587
:0515E200592554FAE553
:0515E7005A3555FBAC74
:0C15EC00568A828B838CF0123547FA245B
:0815F800EC5005755713800249
:021600008A5707
:07160200855D82855E838592
:0A1609005FF0123547FBBB65197551
:0A161300570375580174032FFBE420
:0E161D0038FC89058B828C838DF0EA1233B67F
:07162B000559E4B559020561
:011632005A5D
:0416330085595B85F5
:031637005A5C02F8
:02163A00151089
:0C163C008F82888389F0E55B1233B6A32F
:09164800E55C1233B67582FF2245
:0E16510075AF0390E6C2E0FA43020490E6C2D1
:0E165F00EAF0EA601090E6C2E0FA4302029060
:07166D00E6C2EAF0EA702575
:0916740090E6C2E04402F07A00A5
:03167D00BA0400AC
:0E168000500F90E6C2E054FEF0E0FB4401F093
:03168E000A80ECE3
:0816910090E6C2E0FA4404F007
:0E169900E5807580007582641234F543802070
:0216A7007A00C7
:0316A900BA320052
:0E16AC005025E58030E41390E6C2E090E6C2DF
:0C16BA00E4F0E090E6C2E4F0758201224A
:0D16C600900001C002123508D0020A80D643
:0416D30075820022FA
:0E16D700AA82AB838B9A7C007D008A9B7A00EE
:0216E5007B0088
:0A16E700C3EA954FEB9550501685AD
:0E16F1009C9090E6C2E054FEF0E0FC4401F054
:0716FF000ABA00E40B80E1D0
:0417060075820122C5
:02170A007A0063
:03170C00BA04001C
:0E170F00500F90E6C2E054FEF0E0FB4401F003
:03171D000A80EC53
:0E17200090E6C2E04404F090E6C2E04402F01D
:0A172E0074805580FABA800280042E
:041738007582002294
:04173C00758201228F
:0E366A008F01BF0101010107010003020202EE
:0E36780002000004040404040400000000002A
:0E3686000000003F3911BB1F010101070101C7
:0E369400030100000000000202060606060008
:0E36A20040090F090000003F0802019C0101D1
:0E36B0003F07011000030610010000080C0C7B
:0E36BE000C000000000000000000003F390179
:0E36CC001323AC3F3F0701000103071101006B
:0E36DA00000202020200000000000009360992
:0236E800003FA1
:0E36EA000000000000000000000000000000D2
:0E36F800000000008336040003230302008458
:08370600090202022303020084
:07370E00E0000000EE4E0098
:0E174000C0E0C082C083C002C0D075D000439C
:0C174E00A0015391BF75A2007402551950
:0C175A00FABA02435319FD90E6F3E0FADE
:0E1766004480F00090E6C67484F090E6C774EC
:0E17740009F090E6C87402F090E6C97402F025
:0D17820090E6CA7402F00090E6CEE4F0900C
:0E178F00E6CFF090E6D0F090E6D17401F07550
:04179D00BB00803DD0
:0E17A10090E6F3E0FA4480F00090E6C6748310
:0E17AF00F090E6C77436F090E6C87404F0902F
:0E17BD00E6C9E4F090E6CA7403F00090E6CEB0
:0E17CB00E4F090E6CFF090E6D0F090E6D17416
:0517D90001F075BB06E4
:0E17DE0053A0FED0D0D002D083D082D0E03213
:0E17EC00C0E0C082C083C002C0D075D00043F0
:0E17FA00A0045391BF75A20090E6C2E0FA531E
:0A1808000208BA08054319028049DE
:0E181200C2AF90E6F574FFF000D2AF90E6F39F
:0D182000E0FA4480F00090E6C67484F09079
:0E182D00E6C77409F090E6C87402F090E6C9B0
:0E183B007402F090E6CA7402F00090E6CEE46B
:0E184900F090E6CFF090E6D0F090E6D174017A
:04185700F075BB006D
:0E185B0053A0FBD0D0D002D083D082D0E03298
:0E18690090E60174E6F00090E618E0FA4410F4
:0E187700F00090E61AE0FA4408F00090E6D285
:0E1885007401F00090E6E27402F00090E6D3E9
:0E1893007401F090E6E37401F090E63074808A
:0E18A100F090E6317401F00090E6F574FFF06F
:0E18AF000090370EE49390E6F3F090370FE4CC
:0E18BD009390E6C3F0903710E49390E6C1F0EC
:0E18CB00903711E49390E6C2F0903713E49347
:0618D90090E6C0F07A0069
:0318DF00BA8000CC
:0E18E20050128A037CE4EA90366A93FD8B82F2
:0618F0008C83F00A80E980
:0D18F60090E6C67483F090E6C77436F0905B
:0E190300E6C87404F090E6C9E4F090E6CA74F9
:0E19110003F090E6CB7423F090E6CC7403F064
:0E191F0090E6CD7402F090E60CE4F090E6C67F
:0C192D00F090E6F3E04480F0751900C271
:05193900AF754F407581
:06193E00501775823412FF
:041944002DEC754FC2
:03194800EC7550EB
:0C194B0017758200122DEC90E650740419
:0E195700F090E6607402F0D2AF90E6F3E0FA92
:0E1965004480F00090E6C67483F090E6C774EC
:0E19730036F090E6C87404F090E6C9E4F090F7
:0E198100E6CA7403F00090E6CEE4F090E6CFE4
:0E198F00F090E6D0F090E6D17401F075BB0642
:01199D002227
:0C199E00C2AF75190090E6F574FFF00070
:0E19AA00E5BB30E7FB90371575F08012293A47
:0919B800741CC0E07437C0E01299
:0E19C10033CF15811581D2AF90E6F3E0FA44E2
:0E19CF0080F00090E6C67483F090E6C7743690
:0D19DD00F090E6C87404F090E6C9E4F090C4
:0E19EA00E6CA7403F00090E6CEE4F090E6CF7B
:0E19F800F090E6D0F090E6D17401F075BB06D9
:011A060022BD
:0E1A0700C2AF90E650E4F00090E660E4F0001C
:0D1A150090E6D17401F090E6D37401F090DA
:0D1A2200E6E37401F090E6F574FFF0007546
:0C1A2F00190090E618E0FA54EFF0009067
:0E1A3B00E61AE054F7F0D2AF90371575F08040
:081A490012293A742AC0E0746E
:0B1A510037C0E01233CF158115812251
:07371500494E464F3A200027
:0E371C00677069662061626F727465640A00EE
:0E372A00677069662064656163746976617416
:0437380065640A00BA
:0E1A5C0090E6007410F0758E0075802075B253
:0E1A6A002375900075B3FF75A0C075B4C790CA
:0E1A7800E6C27407F090E6C3E4F090E60B744B
:0E1A860003F00090E610E4F00090E611E4F0AA
:0E1A94000090E61274A0F00090E613E4F0005B
:0E1AA20090E61474E0F00090E615E4F0009079
:0E1AB000E6047480F00090E6047402F00090EA
:0D1ABE00E6047406F00090E604E4F00090E9
:0E1ACB00E6187401F00090E61A7401F0009025
:0E1AD900E68AE4F00090E68BE4F00090E64927
:0E1AE7007482F00090E6497482F00090E649A7
:0E1AF5007482F00090E6497482F00090E6D210
:0E1B03007401F00090E6E27402F00090E680BB
:0D1B1100E0FA30E70E90E6247402F0009038
:061B1E00E625E4F00022C0
:0E1B240090E6247440F00090E6257440F00036
:011B32002290
:0E1B33005380BF43B24090000112350843803A
:051B41004053B2BF2279
:091B4600E582FA700443A040227C
:041B4F0053A0BF22BE
:091B5300E582FA700443A080222F
:041B5C0053A07F22F1
:041B600063A040221C
:041B640063A08022D8
:011B6800225A
:0D1B690090385E7403F090385F7401F075E1
:031B76004F5E754A
:031B79005038756C
:081B7C005102758241022C6840
:0E1B8400AA829038607401F0903861EAF07522
:031B92004F60752C
:031B950050387550
:091B98005102758241122C68759E
:031BA1001BFF2205
:071BA400903862E4F0754F78
:031BAB0062755010
:081BAE003875510175824112E6
:041BB6002C68754FD3
:031BBA0062755001
:081BBD003875510175824112D7
:0E1BC5002BA8903862E0FA530201BA010475B1
:031BD3008201226A
:041BD60075820022F2
:0335780002358099
:0635630075440175386497
:0335930002357B83
:05357B0012280280FE91
:051BDA0090E68BE4F031
:091BDF0090E6A0E0FA20E1F822F2
:031BE8000228EBE5
:031BEB00022911BB
:091BEE00121BDA7402B51D079008
:061BF7003863E4F0A3F0E6
:091BFD00903863E0F50DA3E0F55A
:051C06000E750F407592
:0A1C0B0010E790E6BEE0F5117582C7
:0C1C1500511201D9E5827006751C03F520
:021C210082221D
:0E1C230090E6BEE0FA7B00903863E0FCA3E0A0
:0E1C3100FD903863EA2CF0EB3DA3F0758201C4
:011C3F002282
:0E1C400090E690E0FA8A037A0090E691E07D4B
:091C4E00002AF539ED3BF53A904E
:091C57003849E0FCBC01028003E5
:031C6000021D6BF7
:0E1C630090384AE0FCA3E0FDA3E0FEA3E0FF02
:091C7100EC4D4E4F6003021D2AE8
:0E1C7A0090387FE4F0903845E0FCA3E0FDA335
:0A1C8800E0FEA3E0FFA839A93A7AB4
:0E1C9200007B00C3E89CE99DEA9EEB9F502A70
:0A1CA000E53924F4FAE53A34FFFBBD
:0E1CAA007C007D0090384AEAF0A3EBF0A3EC3A
:0A1CB800F0A3EDF0E53924EAF53958
:081CC200E53A34FFF53A802EEB
:0E1CCA00903845E0FAA3E0FBA3E0FCA3E0FDA8
:0E1CD80090384AEAF0A3EBF0A3ECF0A3EDF095
:0E1CE600903845E0FAA3E0FBA3E0FCA3E0FD8C
:041CF4008A398B3A64
:0C1CF800753B16903845E0FBA3E0FCA310
:0E1D0400E0FDA3E0FEEB24F6FBEC34FFFCED6B
:0E1D120034FFFDEE34FFFE903845EBF0A3ECFD
:0A1D2000F0A3EDF0A3EEF0021E01A7
:081D2A00753B0CE53924F4F5CA
:061D320039E53A34FFF52B
:0C1D38003A90384AE0FBA3E0FCA3E0FD79
:0A1D4400A3E0FEAF39A83AE4F9FA73
:0D1D4E00EF2BFBE83CFCE93DFDEA3EFE907A
:0E1D5B00384AEBF0A3ECF0A3EDF0A3EEF0029B
:021D69001E0159
:0C1D6B00753B00903845E0FAA3E0FBA3B4
:0A1D7700E0FCA3E0FDAE39AF3A78BE
:0E1D8100007900C3EE9AEF9BE89CE99D502A82
:0E1D8F0090384AE0FAA3E0FBA3E0FCA3E0FDDD
:0D1D9D00EE2AFEEF3BFFE83CF8E93DF9902F
:0E1DAA00384AEEF0A3EFF0A3E8F0A3E9F080D2
:011DB80048E2
:0E1DB90090384AE0FAA3E0FBA3E0FCA3E0FDB3
:0E1DC700903845E0FEA3E0FFA3E0F8A3E0F9AA
:0D1DD500EE2AFAEF3BFBE83CFCE93DFD90F7
:0E1DE200384AEAF0A3EBF0A3ECF0A3EDF0908A
:0E1DF0003845E0FAA3E0FBA3E0FCA3E0FD8A87
:031DFE00398B3AE4
:0E1E010090387FE0FAC374808AF063F0809519
:061E0F00F05003021F7CED
:091E1500EA70069038677462F06F
:0C1E1E00903867E0FABA6278AA3B7BF0CB
:061E2A007C007551657596
:031E3000523875B0
:041E3300530085399A
:031E37004F853A9A
:0C1E3A00508A828B838CF01214DBAA8289
:071E4600BA014F750A807517
:031E4D000B3875DA
:061E500008DD75093F7575
:0C1E56000C107582511201A2E58270038D
:031E6200F58222E4
:041E6500754F8075C0
:031E690050387579
:071E6C005100755210E4F56E
:081E73005390386875F000126D
:0E1E7B002A02E5828583F045F060047582003E
:011E89002236
:0E1E8A009038677465F090387F7401F0800620
:061E980090387F74FFF09A
:0C1E9E00903867E0FABA656AAA3B7BF056
:061EAA007C007551657516
:031EB00052387530
:041EB300530085391A
:031EB7004F853A1A
:0C1EBA00508A828B838CF01214DBAA8209
:0C1EC600BA014190386AE090387BF0903F
:0C1ED2003869E0FA90387C75F000EA12E4
:081EDE0033B6903868E0FA9079
:0A1EE600387D75F000EA1233B69063
:091EF000387EE4F5F01233B6125D
:091EF9001651E5827003F5822206
:081F020090387F7401F08006A5
:061F0A0090387F74FFF027
:0C1F1000903865E0FAA3E0FBEA253BF501
:061F1C003BE539C39AF514
:051F220039E53A9BF5D2
:0C1F27003A90384AE0FCA3E0FDA3E0FE85
:0E1F3300A3E0FFE4F8F9EA2CFCEB3DFDE83EEC
:0E1F4100FEE93FFF90384AECF0A3EDF0A3EE6E
:0E1F4F00F0A3EFF0903845E0FCA3E0FDA3E026
:0E1F5D00FEA3E0FFECC39AFAED9BFBEE98F8B2
:0E1F6B00EF99F9903845EAF0A3EBF0A3E8F007
:031F7900A3E9F0E9
:0E1F7C0090387FE0FAC374808AF063F080959D
:061F8A00F0400302204BB1
:081F9000AA3B7BF07C008539BF
:031F98004F853A38
:0C1F9B00508A828B838CF01216D7E582EE
:051FA7007003F5822229
:0E1FAC00903845E0FAA3E0FBA3E0FCA3E0FDC3
:0A1FBA00AE39AF3AE4F8F9EAC39E2D
:0E1FC400FAEB9FFBEC98FCED99FD903845EA96
:0E1FD200F0A3EBF0A3ECF0A3EDF090387BE071
:0C1FE000FAA3E0FBA3E0FCA3E0FDAE3997
:0C1FEC00AF3A7800790090387BEAC39E81
:0E1FF800F0EB9FA3F0EC98A3F0ED99A3F0900E
:0E200600387BE0FAA3E0FBA3E0FCA3E0FDC3FF
:0E201400E49AE49BE49C74808DF063F0809568
:0E202200F0402612170AE582701C90373C75BC
:0A203000F08012293A7444C0E074F5
:0C203A0037C0E01233CF1581158175828C
:02204600002276
:032048007513010C
:04204B007582012277
:0E204F0090E6BCE0FABA020D90E6B8E0FA5353
:07205D000201BA0102800636
:0620640074FE251D50264C
:0A206A00122A82E582600302210AB7
:0A20740090373C75F08012293A7491
:08207E0055C0E07437C0E01208
:0A20860033CF158115817582002209
:0E20900090E6BCE0700D90E6B8E0FA53020155
:05209E00BA01028028D8
:0E20A30090E6BCE0FABA020D90E6B8E0FA53FF
:0720B1000202BA02028013D3
:0E20B80090E6BCE0FABA862E90E6B8E0FA5345
:0520C6000202BA022332
:0E20CB00120350E582703890373C75F0801299
:0720D900293A7462C0E074B3
:0C20E00037C0E01233CF158115817582E6
:0220EC000022D0
:0A20EE0090373C75F08012293A7417
:0820F8006FC0E07437C0E01274
:0A21000033CF15811581758200228E
:04210A0075820122B7
:0E210E0090E6B8E0FABAC00890E6B9E0758233
:02211C0000229F
:0A211E0090E6B8E0FABA4002800330
:032128000221ECA5
:0A212B0090E6B9E0FABA0102801351
:05213500BA0202804126
:05213A00BA0302805B06
:06213F00BA04030221C9ED
:032145000221E88C
:0E214800121BDA90E6BEE0FA24F7500475820E
:02215600002265
:0A215800750F407510E790E6BEE039
:06216200F511750DF87582
:0C2168000E3F7582511201D9E582600320
:032174000221F055
:04217700758200224B
:07217B00121BDA750F40751D
:0621820010E7750DF77572
:092188000E3F7511017582511220
:0921910001D9E5827059F58222A2
:0E219A00121BDA90E6BEE0FA24EF50047582C4
:0221A800002213
:0A21AA00750F407510E790E6BEE0E7
:0621B400F511750DDD754B
:0C21BA000E3F7582511201D9E582702A97
:0321C600F582227D
:0721C900121BDA750F4075CF
:0621D00010E7750DED752E
:0921D6000E3F75110A75825112C9
:0921DF0001D9E582700BF58222A2
:0421E80075820022DA
:0421EC0075820022D6
:0421F00075820122D1
:0421F400750A907563
:0321F8000B38752C
:0621FB0008F775093F75AD
:092201000C017582511201A2903A
:09220A003890E0FA90E00CF0902D
:06221300E064EAF0750A28
:0322190091750BB1
:05221C00387508F8759B
:09222100093F750C087582511289
:04222A0001A27A0093
:03222E00BA0800EB
:0A2231005029EA2491F582E43438C4
:09223B00F583E0FBBBFF027B30E0
:0C2244008A04E4CC25E0CC33FDEC247EC1
:0C225000F582ED34E1F583EBF00A80D25A
:01225C00225F
:05225D009039ABE4F034
:09226200903849E4F03004031245
:02226B0030BA87
:08226D00E5AA30E0030225BAE6
:07227500E51A60030225BA1F
:0A227C0090378675F08012293A743D
:082286008DC0E07437C0E012C6
:0C228E0033CF158115817401B513028057
:01229A00172C
:0E229B00903845E0FAA3E0FBA3E0FCA3E0FDD1
:0922A900EA4B4C4D600302242EA7
:0E22B20090F00175F000123547FA90F00275B9
:0E22C000F000123547FB3395E0FCEBF4FBEC2D
:0E22CE00F4FCEAFD3395E0FEEDB50306EEB537
:0422DC000402800375
:0322E00002240FC6
:0E22E300903844EAF090F000E0FABA01028070
:0122F10003E9
:0322F2000223A91B
:0E22F50090F00475F000123547FBA312354738
:0C230300FCA3123547FDA3123547FE90E5
:0E230F003845EBF0A3ECF0A3EDF0A3EEF09058
:0C231D0038497401F07401B5130280030C
:0323290002242E5D
:0C232C0075130290384AE4F0A3F0A3F00F
:09233800A3F074EF5516F51690A0
:0E234100384EE4F0A3F0A3F0A3F090399DE431
:0E234F00F0A3F090399F740CF0A374F0F0A38B
:08235D00E4F09039ABF07529A2
:032365009D752A39
:0523680038752B009008
:0D236D00399F75F000120957E582600302E8
:02237A00242E0F
:07237C0074204514F51475EF
:0823830013019039ABE4F09066
:0A238B003849F090373C75F08012DD
:07239500293A7494C0E074C2
:0B239C0037C0E01233CF15811581021D
:0223A700242EE2
:0E23A900BA024290399DE0FAA3E0FB4A603789
:0C23B70075130390F00475F00012354718
:0D23C300FAA3123547FBA3123547FCA31205
:0E23D0003547FD903845EAF0A3EBF0A3ECF0A2
:0E23DE00A3EDF090384EE4F0A3F0A3F0A3F0CE
:0223EC0080402F
:0E23EE0090E6A3E04401F090373C75F08012B9
:0723FC00293A74A4C0E0744B
:0C24030037C0E01233CF15811581801F17
:0E240F0090E6A3E04401F090373C75F0801297
:07241D00293A74B8C0E07415
:0A24240037C0E01233CF1581158197
:07242E007402B513028003E4
:032435000225B4C9
:0C2438009039ABE0FA24F650030225B105
:07244400EA2A2A90244B73E1
:07244B000225B10224690221
:0624520024720224A20224
:0624580024D20224FD0263
:06245E00251302251F02F8
:05246400259B0225ACE0
:07246900121B337513010281
:0224700025B491
:04247200750A9D75D5
:032476000B3875AB
:0624790008ED75093F7536
:09247F000C0A7582511201A290B1
:0E24880038A7740AF090399D740BF0A3E4F0AD
:0724960074104516F51675E0
:05249D0013010225B44B
:0424A200750A9D75A5
:0324A6000B38757B
:0624A90008DD75093F7516
:0924AF000C107582511201A2907B
:0E24B80038AD740AF090399D7411F0A3E4F071
:0724C60074104516F51675B0
:0524CD0013010225B41B
:0E24D20074805580FABA800890389D7431F0FD
:0224E000800674
:0624E20090389D7430F0FB
:0E24E80090389E740AF090399D7402F0A3E4BF
:0724F600F07513010225B48B
:0A24FD00121C40E58260030225B4C2
:0725070074104514F5147572
:05250E0013010225B4D9
:07251300121869751A017529
:05251A0013010225B4CD
:04251F007A007B00C3
:0E252300C3EA9414EB940050128A8274F02BD9
:0D253100F5838A04ECF00ABA00E80B80E59F
:0D253E0090F01474FFF090F01574FFF09011
:0E254B00E690E4F090E6917414F012199E9060
:0E255900E6F3E0FA4480F00090E6C67484F0E9
:0D25670090E6C77409F090E6C87402F09089
:0D257400E6C97402F090E6CA7402F000900F
:0D258100E6CEE4F090E6CFF090E6D0F090CA
:0C258E00E6D17401F075BB0075130180EC
:01259A001927
:0D259B0090E6F07455F090E6F174AAF0752A
:0425A8001301800893
:0525AC0075130180031E
:0325B1007513019E
:0625B40090E6497482F07C
:0825BA00E5AA30E503022798B1
:0725C2007403B5130280034E
:0325C9000227984E
:0E25CC0090384EE0FAA3E0FBA3E0FCA3E0FD94
:0925DA00EA4B4C4D60030226910E
:0E25E30090F8007402F0903844E0FA90F8018D
:0E25F10075F000EA1233B6903844E0F4FA9028
:0E25FF00F80275F000EA1233B690F803E4F526
:0E260D00F01233B690399DE0FAA3E0FB8A0488
:0E261B008B057E007F0090F80475F000EC1235
:0A26290033B6A3ED1233B6A3EE1290
:0E26330033B6A3EF1233B690F809E4F5F012B7
:0E26410033B690F80AE4F5F01233B690F80BB9
:0E264F00E4F5F01233B690E680E0FC30E725AB
:0E265D00C374F49A74019BB3E433FCC3743865
:0E266B009AE49BB3E433FA4C600D90F80875C6
:09267900F00074011233B680096F
:0926820090F808E4F5F01233B6FB
:06268B00753C0CE4F53D76
:0C26910090384EE0A3E0A3E0A3E0AA3CD8
:02269D00AB3D53
:0E269F00C002C00390384EE0FCA3E0FDA3E0B3
:0D26AD00FEA3E0FF90399DE0FAA3E0FB8A58
:0426BA003E8B3F759F
:0726BE004000754100C3E577
:0626C5003E9CE53F9DE58F
:0A26CB00409EE5419FE433D003D0A8
:0626D50002600302275C15
:0926DB008A048B050ABA00010B08
:0826E4008C4274F82DF54390BF
:0E26EC00384EE0FEA3E0FFA3E0A3E0FDEE24E5
:0A26FA009DF582EF3438F583E0858A
:0A2704004282854383F090E680E0F6
:0E270E00FC30E71E90399DE0FCA3E0FDE4BC2A
:06271C000004BD020104EF
:09272200FEE4BC4004BD0001040A
:05272B004E6002802C4D
:0E27300090384EE0FCA3E0FDA3E0FEA3E0FF26
:0D273E000CBC00090DBD00050EBE00010F12
:0E274B0090384EECF0A3EDF0A3EEF0A3EFF00B
:0327590002269FB6
:0C275C0090E698EBF090E699EAF0E4F5C6
:042768003CF53D906F
:0E276C00384EE0FAA3E0FBA3E0FCA3E0FDC3BF
:08277A00EA953EEB953FEC955A
:0727820040ED954140107588
:07278900130174EF5516F572
:082790001690399DE4F0A3F05E
:09279800E51B7005F582121B849B
:0627A1007538640222629B
:0C27A700C021C0E0C0F0C082C083C002AE
:0E27B300C003C004C005C006C007C000C001BE
:0A27C100C0D075D0001544E5447047
:0827CB0009754432121B607510
:0227D3001B00E9
:0827D5007401B51D09151EE594
:0627DD001E7003123082A1
:0E27E300C2CFD0D0D001D000D007D006D00594
:0E27F100D004D003D002D083D082D0F0D0E04C
:0327FF00D02132B4
:07280200121A5C121B69129F
:0628090002A31214D375B6
:0C280F001A0012284E90E601E04404F08C
:09281B00C2AF1221F4122E3E128C
:052824002FB97AA77B2B
:0B282900278A828B831234D8D2AF12B2
:0E2834001BA4E5826008758204121B848006D6
:06284200758202121B84E6
:062848001229DE02225DF0
:08373C004552524F523A2000A1
:0E37440066696E616C697A696E67204650474F
:03375200410A0029
:0D37550064667520726571756573740A00F5
:0D376200746D6320726571756573740A00E3
:0E376F00696E76616C696420636C617373200F
:09377D00726571756573740A0030
:07378600494E464F3A2000B6
:07378D006C6F63616C0A0020
:0E37940073796E746178206661696C75726578
:0237A2000A001B
:0E37A400756E6B6E6F776E206D657373616767
:0637B200652049440A00F5
:0E37B8006254616720696E76616C69640A0074
:0A284E00C2ACC2009039ACE4F09077
:0828580039ADF09039AEF090AB
:0E28600039AFF090E6087401F07598501099A9
:03286E00028000E5
:05287100109802800038
:04287600754F8575A0
:06287A00502875822312B4
:052880002D37D2AC224F
:0E288500C0E0C082C083C002C003C0D075D0C6
:0828930000C2AC10980280178E
:0C289B009039AEE0FA9039AE04F0EA2467
:0A28A700B0F582E4343AF583E599B8
:0128B100F036
:0528B2001099028025D1
:0E28B7009039ACE0FA9039ADE0FBEAB50304CD
:0428C500C2008013BA
:0C28C9009039ADEB04F0EB24B0F582E494
:0728D5003439F583E0F599A9
:0E28DC00D2ACD0D0D003D002D083D082D0E0D6
:0128EA0032BB
:0C28EB00AA82C2AC3000189039ACE0FBAF
:0C28F7009039AC04F0EB24B0F582E4341E
:0729030039F583EAF08004BE
:04290A00D2008A99D4
:03290E00D2AC2226
:0E2911009039AEE0FA9039AFE0FBEAB5030270
:02291F00801422
:0C2921009039AFEB04F0EB24B0F582E439
:08292D00343AF583E0FA800260
:022935007A0026
:032937008A82226F
:06293A00AA82AB83ACF0A1
:0E2940008A828B838CF0123547FD60188D82E1
:05294E000ABA00010BB4
:0E295300C002C003C0041228EBD004D003D091
:032961000280DC15
:012964002250
:0E2965007A009039AEE0FB9039AFE0FCEBB5A4
:0429730004028002D8
:022977007A01E3
:032979008A82222D
:08297C0085825285835385F02A
:0429840054AD4FAE51
:0429880050AF51A853
:04298C0052A953AA4F
:0129900054F2
:0E2991008D828E838FF0123547FBA3AD82AE90
:0E299F0083888289838AF0EB1233B6A3A88264
:0A29AD00A983EB70DF855282855389
:0529B700838554F022AD
:0829BC0090E6A0E04401F022C6
:0E29C400AA8274805AC423541FFB740F5A90C9
:0C29D200E6834BF090E683E04420F02206
:0E29DE0090E680E0440AF09000FA123508906E
:0E29EC00E65D74FFF090E65F74FFF05391EF2C
:0829FA0090E680E054F7F022A2
:0A2A0200AA82AB83ACF0E552455305
:062A0C007004900000229E
:052A1200AD4FAE50AF16
:042A170051A852A9C7
:012A1B005367
:052A1C0018B8FF0119CC
:0E2A2100E84960378A828B838CF0123547F5C6
:0A2A2F0054E5546028C000C0018D7A
:0C2A3900828E838FF0123547F8B55404EC
:042A45007401800197
:012A4900E4A8
:0B2A4A00D001D000600C0ABA00010BA4
:072A55000DBD00C30E80C09F
:0E2A5C008A828B838CF0123547FA3395E0FBAB
:0E2A6A008D828E838FF0123547FD3395E0FC90
:0A2A7800EAC39DF582EB9CF5832272
:06358D00E478FFF6D8FD12
:07356900751C00751D0075C3
:023570001EFF3C
:0E2A820090E6B8E0FA530280BA805F90E6B9A1
:072A9000E0FABA0202800A1D
:052A9700BA0302800BF0
:052A9C00BA054980337A
:062AA100E51C7582002215
:0C2AA70090E740E51CF090E741E4F0905F
:0D2AB300E742F090E74374FFF090E744E540
:0C2AC0001DF090E745E4F090E68AF090ED
:082ACC00E68B7406F0022BA456
:0C2AD40090E740E51DF090E68AE4F090E9
:082AE000E68B7401F0022BA447
:042AE80075820022D1
:0B2AEC0090E6B8E0FA30E703022BA0F0
:0C2AF70090E6B9E0FA6013BA01028025F5
:052B0300BA040280612C
:062B0800BA0603022B7D5A
:032B0E00022B99FE
:082B1100E51D700C1230827505
:062B19001D01751EFF0204
:022B1F002BA4E5
:072B2100751C0F75820022F4
:072B28007402B51D028005D7
:052B2F007405B51D1B3B
:0E2B340090E6BEE06015121BEEE5827009759A
:082B42001C03751D0AF5822237
:052B4A00751D0580551A
:0C2B4F007405B51D0E90E6BEE070081283
:072B5B003082751D08804265
:072B6200751C0F75820022B3
:092B6900740AB51D08751C007505
:042B72001D02802E92
:072B7600751C0F758200229F
:062B7D00E4B51D02800F0B
:072B83007401B51D0280087A
:082B8A00751C00751D0280128C
:072B9200751C0F7582002283
:072B9900751C0F758200227C
:042BA0007582002218
:042BA4007582012213
:0A2BA800AA82E55170047582012233
:0E2BB20090E678E0FB20E6F890E6787480F07C
:0A2BC000EA2AFA90E67974014AF05F
:0E2BCA0090E678E0FA30E0F890E678E0FA3035
:052BD800E203022C5D88
:0B2BDD0090E678E0FA20E103022C5D96
:0C2BE8007401B5510890E678E0FA442032
:012BF400F0F0
:092BF50090E679E0F552AA4FAB1D
:032BFE0050AC5187
:042C0100DC02803041
:0E2C050090E678E0FD30E0F890E678E0FD2003
:0D2C1300E248BC010890E678E0FD4420F0A6
:0E2C200090E679E0FD8A828B83F0A3AA82AB56
:072C2E00838A4F8B5080CC1C
:0E2C350090E678E0FA30E0F890E678E0FA20D9
:0C2C4300E21890E678E04440F0AA4FABA5
:0C2C4F005090E679E08A828B83F0758259
:022C5B00012254
:0B2C5D0090E678E04440F07582002211
:022C6800AA823E
:0E2C6A0090E678E0FB20E6F890E6787480F0C3
:072C7800EA2AFA90E679F068
:0E2C7F0090E678E0FA30E0F890E678E0FA208F
:0C2C8D00E24790E678E0FA30E13FAA4F01
:042C9900AB50AC513F
:0E2C9D00EC602B8A828B83E0FDA3AA82AB83BE
:062CAB0090E679EDF01C3B
:0E2CB10090E678E0FD30E0F890E678E0FD2057
:0C2CBF00E21590E678E0FD20E1D4800BE7
:0B2CCB0090E678E04440F075820122A2
:0B2CD60090E678E04440F07582002298
:082CE10085825285835385F0C2
:042CE90054AD52AEE6
:032CED0053AF548E
:0E2CF0008D828E838FF012354760070DBD0078
:042CFE00F10E80EE65
:052D0200A84FA950AA32
:052D0700518E048F0352
:0E2D0C00888289838AF0123547FEA3A882A927
:0E2D1A00838D828C838BF0EE1233B6A3AD82D4
:0A2D2800AC83EE70DF855282855304
:052D3200838554F0222E
:052D3700AA82BA0300AE
:072D3C004005EA249C500150
:012D4300226D
:092D4400740F5AFBBB0302800767
:072D4D00740F5AFBBB0B459C
:0A2D5400A2AF9201C2AFEA2400F51D
:0C2D5E0082E43400F5837402F07B007402
:0C2D6A00012AFCE43BFDEC2400F582EDA6
:0A2D76003400F583E550FCF0740210
:0C2D80002AFAE43BFBEA2400F582EB3465
:0A2D8C0000F583AA4F7B00EAF0A2D5
:032D96000192AFF8
:012D99002217
:082D9A00E582FA2483500122B6
:072DA20074035AFB600122DB
:0A2DA900A2AF9202C2AFEA2400F5C7
:0C2DB30082E43401F5837402F07B0074AC
:0C2DBF00012AFCE43BFDEC2400F582ED51
:0A2DCB003401F583E550F074022A8C
:0B2DD500FAE43BFBEA2400F582EB343B
:082DE00001F583AA4FEAF0A2FD
:042DE8000292AF2282
:082DEC00E582FA24CB5001221C
:072DF40074035AFB60012289
:0A2DFB00A2AF9203C2AFEA2480F5F4
:0C2E050082E43400F5837402F07B00745A
:0C2E1100012AFCE43BFDEC2480F582ED7E
:0A2E1D003400F583E550F074022A3A
:0B2E2700FAE43BFBEA2480F582EB3468
:082E320000F583AA4FEAF0A2AB
:042E3A000392AF222E
:082E3E00C2E8C2EA754F0075FD
:062E4600500175824312E9
:042E4C002D37754F5A
:032E50008075503A
:0C2E530000758253122D370090E650E409
:0E2E5F00F00090E652E4F00090E654E4F0003B
:0E2E6D0090E656E4F00090E65174FFF00090FD
:0E2E7B00E65374FFF00090E65574FFF00090EF
:0E2E8900E65774FFF00090E658E4F090E6592A
:0E2E970074FFF090E65AE4F090E65B74FFF0F2
:0E2EA50090E65CE4F090E65D74FFF090E65E6F
:0E2EB300E4F090E65F74FFF00090E660E4F05B
:0D2EC1000090E66174FFF090E662E4F0908E
:0E2ECE00E66374FFF090E665E4F090E6687449
:0A2EDC000BF05391AFD2E8D2EA22C6
:06357200754500754600DE
:0A2EE60090E680E0FA30E719754726
:032EF00000754822
:032EF300E075493E
:032EF60012754A08
:032EF900E0754B36
:032EFC001C754CF6
:032EFF00E0754D2E
:032F020074754E95
:022F0500E022C8
:042F0700754758753D
:032F0B0048E07526
:032F0E00496A7598
:032F11004AE0751E
:032F14004B747586
:032F17004CE07516
:032F1A004D1C75D6
:032F1D004EE02261
:092F20005391EF75A100D20432B7
:0C2F2900C021C0E0C0F0C082C083C00224
:0E2F3500C003C004C005C006C007C000C00134
:0E2F4300C0D075D0005391EF75A100122EE69C
:0C2F5100751D00D0D0D001D000D007D0FA
:0E2F5D0006D005D004D003D002D083D082D09D
:062F6B00F0D0E0D021329D
:0C2F7100C021C0E0C0F0C082C083C002DC
:0E2F7D00C003C004C005C006C007C000C001EC
:0E2F8B00C0D075D0005391EF75A100122EE654
:0C2F9900751D00D0D0D001D000D007D0B2
:0E2FA50006D005D004D003D002D083D082D055
:062FB300F0D0E0D0213255
:052FB900122EE6754F29
:032FBE002075502B
:082FC1002F758200122D9A7594
:032FC9004F297518
:062FCC00502F7582101267
:042FD2002D9A754F70
:032FD600717550C2
:0C2FD9002F758214122D9A90E65C743162
:022FE500F022D8
:0D2FE700E582547FFA24F750047582002221
:072FF400BA010475820122FD
:082FFB00530201E4BA000104D5
:03300300F5822231
:09300600AA82BA010490E6A1229D
:07300F00BA810490E6A22241
:0A30160053027FEA700490E6A02246
:0D302000EAC31324A2F582E434E6F583220E
:04302D007547A675C8
:0330310048E075FF
:033034004BB87521
:033037004CE02248
:0C303A00C021C0E0C0F0C082C083C00212
:0E304600C003C004C005C006C007C000C00122
:0E305400C0D075D0005391EF75A10012302D41
:0C306200751D02D0D0D001D000D007D0E6
:0E306E0006D005D004D003D002D083D082D08B
:06307C00F0D0E0D021328B
:06308200E51D7018754FFA
:033088003A755046
:08308B0030758210122D9A75B8
:033093004F3A753C
:06309600503075821402A7
:02309C002D9A6B
:04309E00754F2975CC
:0630A200502F7582101290
:0430A8002D9A754F99
:0330AC00717550EB
:0830AF002F758214122D9A7591
:0330B7001D0022D7
:0C30BA00C20490E6B8E0FA530260BA00CD
:0330C6000280384D
:0530C900BA2002800D99
:0530CE00BA4002801E63
:0530D300BA6002801349
:0330D8000233AE12
:0A30DB0012204FE58260030233AEBD
:0630E5001229BC0233AE0B
:0630EB001229BC0233AE05
:0A30F10012210EE58260030233AEE7
:0630FB001229BC0233AEF5
:0D31010090E6B8E0FA530280BA8002800325
:03310E000232A8E2
:0B31110090E6B9E0FABA000302321F9A
:05311C00BA0602803537
:05312100BA080280085D
:05312600BA0A02801747
:03312B000232A2CB
:0C312E0090E740E545F090E68AE4F09060
:08313A00E68B7401F00233AED4
:0C31420090E740E546F090E68AE4F0904B
:08314E00E68B7401F00233AEC0
:0A31560090E6BBE0FABA0102801D0A
:05316000BA0202803EEE
:05316500BA0302805FC7
:05316A00BA06028021FD
:05316F00BA07028042D6
:06317400BA210302320241
:03317A0002321905
:0A317D00AA47AB4890E6B3EBF07BE5
:093187000090E6B4EAF00233AE58
:0A319000AA49AB4A90E6B3EBF07BCE
:09319A000090E6B4EAF00233AE45
:0A31A300AA4BAB4C90E6B3EBF07BB7
:0931AD000090E6B4EAF00233AE32
:0A31B600AA4DAB4E90E6B3EBF07BA0
:0931C0000090E6B4EAF00233AE1F
:0E31C90090E6BAE0FA90E0D3E0FBC3EA9B4048
:0731D700061229BC0233AE11
:0C31DE0090E6BAE075F002A424D4F5825B
:0B31EA0074E035F0F583E0FAA3E090FC
:0D31F500E6B3F07B0090E6B4EAF00233AEE2
:0A3202007ACA7BE090E6B3EBF07AA5
:0A320C00CA7BE07B0090E6B4EAF014
:033216000233AED2
:063219001229BC0233AED5
:0D321F0090E6B8E0FA53021FBA0002800AE0
:05322C00BA0102801D43
:05323100BA0268802EC6
:0E32360090E7407401F090E741E4F090E68AE2
:0A324400F090E68B7402F00233AE46
:0E324E0090E740E4F090E741F090E68AF090BF
:08325C00E68B7402F00233AEB0
:0E32640090E6BCE0F582122FE7E5826025902F
:0E327200E6BCE0F582123006E0FA530201904D
:0E328000E740EAF090E741E4F090E68AF09033
:08328E00E68B7402F00233AE7E
:063296001229BC0233AE58
:06329C001229BC0233AE52
:0632A2001229BC0233AE4C
:0C32A80090E6B9E0FA24F450030233ABC6
:0732B400EA2A2A9032BB73E5
:0732BB000233AB0232F10205
:0632C200337302335402D5
:0632C80033AB0233AB0240
:0632CE0033AB0233AB023A
:0632D40033AB0232DF0201
:0532DA0033AB0232E8F5
:0932DF0090E6BAE0F5450233AEB9
:0932E80090E6BAE0F5460233AEAF
:0D32F10090E6B8E0FA53021FBA0002800513
:0532FE00BA024E800A37
:0A33030090E6BAE01229BC0233AED6
:0D330D0090E6BAE0703790E6BCE0F5821261
:0D331A002FE7E582602A90E6BCE0F5821204
:0E3327003006AA82AB83E0FC5304FE8A828B40
:0E33350083ECF090E6A3E054FEF090E6BCE0DE
:07334300F5821229C4806429
:05334A001229BC805FA8
:05334F001229BC805AA8
:0E33540090E6B8E0FA53021FBA004F90E6BAB6
:07336200E0FABA0102800548
:05336900BA02028040E1
:05336E001229BC803BA8
:0E33730090E6BAE0FA702C90E6BCE0F582120B
:0D3381002FE7E582601A90E6BCE0F58212AD
:0E338E003006AA82AB83E0FC4304018A828BE6
:05339C0083ECF0800D40
:0533A1001229BC8008A8
:0533A6001229BC8003A8
:0333AB001229BC28
:0833AE0090E6A0E04480F0224B
:0E33B60020F71030F6118883A88220F507F664
:0533C400A883758300E1
:0133C90022E1
:0333CA00F280F797
:0233CD00F022EC
:0533CF00C01F85811FF5
:0B33D400E51F24FDF886831886821890
:0E33DF00E493A324DB600C242560051234BDAA
:0233ED0080F06E
:0333EF000234D5D0
:0933F200D2D5E493A3C083C0828C
:0333FB00B4731494
:0933FE0086F018868318868218F7
:0B3407001235476054A31234BD80F55D
:0B341200B4630818E6181234BD8043B4
:0E341D00B46417E630E74618E6F42401F6081A
:0C342B00E6F43400F6742D1234BD80333A
:0A343700B4782D868318868218E40D
:0B3441001234AEE5831234ADE58312B7
:0A344C0034AEE5821234ADE58212C1
:0A34560034AE30D50574301234BDD9
:07346000D082D0830233DFAC
:03346700B475F643
:06346A00E6FA18E6F9186D
:0D3470007C107D27123498FF7CE87D03124C
:0E347D003498C4F5837C647D00123498428339
:0D348B00E975F00A84C445F0F582EF80A9D0
:023498007B00B7
:0E349A000BC3E99CF9EA9DFA50F61BE92CF9E8
:0534A800EA3DFAEB22F1
:0134AD00C45A
:0734AE00540F700320D51F2D
:0834B500C2D52490D43440D4A8
:0E34BD00C083C082C0F0F582E8C0E0121BE8B8
:0934CB00D0E0F8D0F0D082D083EB
:0134D40022D5
:0334D500D01F22E3
:0A34D800AA82AB83C2AD8A4F8B506D
:0E34E20075822B122D3775CB6375CAC075C865
:0434F00004D2AD2233
:0134F40022B5
:0234F500AA82A9
:0634F7001234F4DAFB229E
:0334FD0090FB50F1
:08350000A3E582458370F92266
:04350800AA82AB8365
:08350C001234FD1ABAFF011B85
:07351400BA00F5BB00F22232
:05351B00AA82BA410084
:0B3520004009EA24A540047582012246
:04352B007582002283
:04352F00AA82AB833E
:083533001235476003A380F884
:0C353B00C3E5829AF582E5839BF58322AC
:03358000758162F0
:0A358300120180E582600302357B2F
:0E35470020F71430F6148883A88220F507E6DA
:06355500A883758300222B
:03355B00E280F714
:03355E00E49322D1
:02356100E02266
:00000001FF
